:020000040000FA
:0A0000000000000025EF00F033D0EF
:0800180087D0056A046EFF0E9B
:100020000426052200D0D8A01200030E036EE60EAF
:1000300002D8F5D7036AFE0F026EE86A035AD8A009
:1000400012000000020600D0F8D74F0EAF6E240E4B
:10005000AC6E900EAB6E0001C69A400E926EE00E32
:10006000936EC00E946E0F0EC16E070EB46E73D0F9
:100070009EAA1BD0060EAB1412E1E2CF3BF0E1CFFB
:100080003AF03C2A11EE00F03C50E126000EE2224C
:10009000AECFE7FF3BC0E2FF3AC0E1FF1100AE5038
:1000A000AE50AB98AB8811000AD0F2A408D0F294FD
:1000B000084A092A817A076AD6CF06F01100110092
:1000C0003C503D5C14E03D2AEACF03F0E9CF02F05A
:1000D00001EE00F03D50E926000EEA22EF50026EDC
:1000E00003C0EAFF02C0E9FFD880120004D0E8682C
:1000F000026ED8A0120012003C6A3D6A9D8A9F8A57
:10010000F28EF28C12009D9A01EE00F0010EF46E58
:10011000F36AF306000EF45AEE6AF450F310F9E1B4
:100120003C6A3D6A9D8A1200F29EE0CFB6FDD8CFB0
:10013000B7FDE8CFB8FDF28E0001A192F29EB6CDD8
:10014000E0FFB7CDD8FFB8CDE8FFF28E10009EA833
:10015000FED7AD6E120093948A94929089909292F9
:100160008992929489949296899692988998929A73
:10017000899A94908B9094928B9294948B94949669
:100180008B9694988B98949A8B9A939A8A9A1C6AD5
:100190005CEC0BF059EC0DF0236A226A256A246AA4
:1001A000276A266A296A286A2B6A2A6A2D6A2C6AB3
:1001B0002F6A2E6A316A306A336A326A356A346A63
:1001C000376A366A396A386A939A8A8A320E25DF24
:1001D000939A8A9A1B6A1A6A216A206A8DDF93DFD2
:1001E000CD6AF294F28A870ED56EB16AA192A0828E
:1001F000D08EA292B00EB16E63DF0A6EBE0E0A5CA4
:1002000009E3FE0E0A5C03E3BAEF04F003D00C6AC4
:10021000BAEF04F00AAE22D00C6A8D0E0A5C05E13A
:100220000AC00CF00D680E6817D09D0E0A5C05E13F
:100230000AC00CF00F6810680FD0AD0E0A5C05E123
:100240000AC00CF01168126807D0BD0E0A5C04E108
:100250000AC00CF013681468BAEF04F00C5204E101
:10026000BAEF04F0BAEF04F08D0E0C5CD8A460D0A5
:100270000D2803E10AC00DF057D0330E0D5C04E1E8
:100280001A908B9A20904FD0370E0D5C04E11A9291
:100290008B98209248D0390E0D5C03E0450E0D5C22
:1002A00004E11A948B9620943ED03C0E0D5C04E140
:1002B0001A968B94209637D0410E0D5C04E11A9863
:1002C0008B92209830D0430E0D5C04E11A9A8B90EB
:1002D000209A29D0440E0D5C04E11A9C899A209C36
:1002E00022D0480E0D5C04E11A9E8998209E1BD0F6
:1002F000550E0D5C04E11B908996219014D0570E89
:100300000D5C04E11B92899421920DD0580E0D5C76
:1003100004E11B948992219406D0590E0D5C03E1EF
:100320001B96899021960D68BAEF04F0BAEF04F09D
:100330009D0E0C5CD8A4A0EF04F00F2804E10AC0C5
:100340000FF09EEF04F00AC010F01052D8A459D05C
:10035000330E0F5C04E11A908B9A20904FD0370E29
:100360000F5C04E11A928B98209248D0390E0F5CF2
:1003700003E0450E0F5C04E11A948B9620943ED066
:100380003C0E0F5C04E11A968B94209637D0410EF8
:100390000F5C04E11A988B92209830D0430E0F5CCA
:1003A00004E11A9A8B90209A29D0440E0F5C04E144
:1003B0001A9C899A209C22D0480E0F5C04E11A9E58
:1003C0008998209E1BD0550E0F5C04E11B908996E6
:1003D000219014D0570E0F5C04E11B928994219256
:1003E0000DD0580E0F5C04E11B948992219406D025
:1003F000590E0F5C03E11B96899021960F68BAEFA6
:1004000004F01C52D8B49DEF04F0330E0F5C35E1BC
:10041000225202E12352D8A4208000011A80D7CFB3
:1004200007F0D6CF06F001EEB6F0D8901034E926EA
:10043000000EEA22EECF00F0EFCF01F001C03FF056
:1004400000C03EF03EC000F03FC001F00050062466
:10045000166E01500720176E000E0820186E000E51
:100460000920196E19C057F018C056F017C06FF068
:1004700016C06EF08B8A9DEF04F0370E0F5C35E1ED
:10048000245202E12552D8A4208200011A82D7CF3B
:1004900007F0D6CF06F002EEB6F0D8901034E92679
:1004A000000EEA22EECF00F0EFCF01F001C041F0E4
:1004B00000C040F040C000F041C001F000500624F0
:1004C000166E01500720176E000E0820186E000EE1
:1004D0000920196E19C059F018C058F017C071F0F2
:1004E00016C070F08B889DEF04F0390E0F5C03E0AE
:1004F000450E0F5C34E1265202E12752D8A4208435
:1005000000011A84D7CF07F0D6CF06F003EEB6F07D
:10051000D8901034E926000EEA22EECF00F0EFCF9B
:1005200001F001C043F000C042F042C000F043C0FF
:1005300001F000500624166E01500720176E000EC1
:100540000820186E000E0920196E19C05BF018C043
:100550005AF017C073F016C072F08B86EED13C0EC5
:100560000F5C34E1285202E12952D8A42086000110
:100570001A86D7CF07F0D6CF06F004EEB6F0D890A3
:100580001034E926000EEA22EECF00F0EFCF01F0A2
:1005900001C045F000C044F044C000F045C001F087
:1005A00000500624166E01500720176E000E08201A
:1005B000186E000E0920196E19C05DF018C05CF0AD
:1005C00017C075F016C074F08B84B7D1410E0F5C64
:1005D00034E12A5202E12B52D8A4208800011A8863
:1005E000D7CF07F0D6CF06F005EEB6F0D89010348E
:1005F000E926000EEA22EECF00F0EFCF01F001C0B5
:1006000047F000C046F046C000F047C001F000507F
:100610000624166E01500720176E000E0820186E73
:10062000000E0920196E19C05FF018C05EF017C0E7
:1006300077F016C076F08B8280D1430E0F5C34E1E8
:100640002C5202E12D52D8A4208A00011A8AD7CF59
:1006500007F0D6CF06F006EEB6F0D8901034E926B3
:10066000000EEA22EECF00F0EFCF01F001C049F01A
:1006700000C048F048C000F049C001F00050062416
:10068000166E01500720176E000E0820186E000E1F
:100690000920196E19C061F018C060F017C079F018
:1006A00016C078F08B8049D1440E0F5C34E12E5295
:1006B00002E12F52D8A4208C00011A8CD7CF07F06A
:1006C000D6CF06F007EEB6F0D8901034E926000E2B
:1006D000EA22EECF00F0EFCF01F001C04BF000C0F6
:1006E0004AF04AC000F04BC001F000500624166EDC
:1006F00001500720176E000E0820186E000E09200A
:10070000196E19C063F018C062F017C07BF016C0F4
:100710007AF0898A12D1480E0F5C34E1305202E13E
:100720003152D8A4208E00011A8ED7CF07F0D6CF31
:1007300006F008EEB6F0D8901034E926000EEA2252
:10074000EECF00F0EFCF01F001C04DF000C04CF053
:100750004CC000F04DC001F000500624166E015050
:100760000720176E000E0820186E000E0920196E63
:1007700019C065F018C064F017C07DF016C07CF099
:100780008988DBD0550E0F5C34E1325202E13352DE
:10079000D8A4218000011B80D7CF07F0D6CF06F068
:1007A00009EEB6F0D8901034E926000EEA22EECF1A
:1007B00000F0EFCF01F001C04FF000C04EF04EC08E
:1007C00000F04FC001F000500624166E01500720C3
:1007D000176E000E0820186E000E0920196E19C041
:1007E00067F018C066F017C07FF016C07EF08986EB
:1007F000A4D0570E0F5C34E1345202E13552D8A434
:10080000218200011B82D7CF07F0D6CF06F00AEE77
:10081000B6F0D8901034E926000EEA22EECF00F0B0
:10082000EFCF01F001C051F000C050F050C000F017
:1008300051C001F000500624166E01500720176EBB
:10084000000E0820186E000E0920196E19C069F0FC
:1008500018C068F017C081F016C080F089846DD090
:10086000580E0F5C34E1365202E13752D8A421848D
:1008700000011B84D7CF07F0D6CF06F00BEEB6F001
:10088000D8901034E926000EEA22EECF00F0EFCF28
:1008900001F001C053F000C052F052C000F053C04C
:1008A00001F000500624166E01500720176E000E4E
:1008B0000820186E000E0920196E19C06BF018C0C0
:1008C0006AF017C083F016C082F0898236D0590EC4
:1008D0000F5C33E1385202E13952D8A4218600017D
:1008E0001B86D7CF07F0D6CF06F00CEEB6F0D89027
:1008F0001034E926000EEA22EECF00F0EFCF01F02F
:1009000001C055F000C054F054C000F055C001F0D3
:1009100000500624166E01500720176E000E0820A6
:10092000186E000E0920196E19C06DF018C06CF019
:1009300017C085F016C084F089800F681BD01AD0CC
:10094000AD0E0C5C0BE1112803E10AC011F004D0DC
:100950000AC012F0F8EC09F00DD00CD0BD0E0C5C02
:1009600009E1132803E10AC013F004D00AC014F00F
:10097000ECEC0AF01AA039D056C018F057C019F0A4
:100980006EC016F06FC017F0D7CF07F0D6CF06F0C5
:100990001650065C17500758185008581950095837
:1009A00023E38B9A1A9020A01FD0225202E12352F7
:1009B0001AE0D7CF07F0D6CF06F022500624166EE5
:1009C00023500720176E000E0820186E000E092015
:1009D000196E19C087F018C086F017C09FF016C0B6
:1009E0009EF0000101D0209033D020A030D086C0EE
:1009F00018F087C019F09EC016F09FC017F0D7CF2F
:100A000007F0D6CF06F01650065C1750075818505E
:100A10000858195009581AE31A803EC000F03FC028
:100A200001F000500624166E01500720176E000ECC
:100A30000820186E000E0920196E19C057F018C052
:100A400056F017C06FF016C06EF08B8A01D08B9AEB
:100A50001AA239D058C018F059C019F070C016F059
:100A600071C017F0D7CF07F0D6CF06F01650065C4E
:100A700017500758185008581950095823E38B98F5
:100A80001A9220A21FD0245202E125521AE0D7CF99
:100A900007F0D6CF06F024500624166E2550072006
:100AA000176E000E0820186E000E0920196E19C06E
:100AB00089F018C088F017C0A1F016C0A0F000019E
:100AC00001D0209233D020A230D088C018F089C045
:100AD00019F0A0C016F0A1C017F0D7CF07F0D6CFFD
:100AE00006F01650065C1750075818500858195051
:100AF00009581AE31A8240C000F041C001F00050CA
:100B00000624166E01500720176E000E0820186E7E
:100B1000000E0920196E19C059F018C058F017C0FE
:100B200071F016C070F08B8801D08B981AA439D060
:100B30005AC018F05BC019F072C016F073C017F0FD
:100B4000D7CF07F0D6CF06F01650065C17500758DF
:100B5000185008581950095823E38B961A9420A46A
:100B60001FD0265202E127521AE0D7CF07F0D6CF86
:100B700006F026500624166E27500720176E000E2A
:100B80000820186E000E0920196E19C08BF018C0CD
:100B90008AF017C0A3F016C0A2F0000101D0209483
:100BA00033D020A430D08AC018F08BC019F0A2C076
:100BB00016F0A3C017F0D7CF07F0D6CF06F0165027
:100BC000065C1750075818500858195009581AE36E
:100BD0001A8442C000F043C001F000500624166E93
:100BE00001500720176E000E0820186E000E092015
:100BF000196E19C05BF018C05AF017C073F016C018
:100C000072F08B8601D08B961AA639D05CC018F092
:100C10005DC019F074C016F075C017F0D7CF07F09B
:100C2000D6CF06F01650065C1750075818500858D3
:100C30001950095823E38B941A9620A61FD02852E6
:100C400002E129521AE0D7CF07F0D6CF06F028509C
:100C50000624166E29500720176E000E0820186E05
:100C6000000E0920196E19C08DF018C08CF017C045
:100C7000A5F016C0A4F0000101D0209633D020A624
:100C800030D08CC018F08DC019F0A4C016F0A5C0EB
:100C900017F0D7CF07F0D6CF06F01650065C1750E6
:100CA000075818500858195009581AE31A8644C0B2
:100CB00000F045C001F000500624166E01500720D8
:100CC000176E000E0820186E000E0920196E19C04C
:100CD0005DF018C05CF017C075F016C074F08B841E
:100CE00001D08B941AA839D05EC018F05FC019F0FB
:100CF00076C016F077C017F0D7CF07F0D6CF06F042
:100D00001650065C175007581850085819500958C3
:100D100023E38B921A9820A81FD02A5202E12B526B
:100D20001AE0D7CF07F0D6CF06F02A500624166E69
:100D30002B500720176E000E0820186E000E092099
:100D4000196E19C08FF018C08EF017C0A7F016C02A
:100D5000A6F0000101D0209833D020A830D08EC05A
:100D600018F08FC019F0A6C016F0A7C017F0D7CFA3
:100D700007F0D6CF06F01650065C175007581850EB
:100D80000858195009581AE31A8846C000F047C09D
:100D900001F000500624166E01500720176E000E59
:100DA0000820186E000E0920196E19C05FF018C0D7
:100DB0005EF017C077F016C076F08B8201D08B9270
:100DC0001AAA39D060C018F061C019F078C016F0C6
:100DD00079C017F0D7CF07F0D6CF06F01650065CD3
:100DE00017500758185008581950095823E38B908A
:100DF0001A9A20AA1FD02C5202E12D521AE0D7CF06
:100E000007F0D6CF06F02C500624166E2D50072082
:100E1000176E000E0820186E000E0920196E19C0FA
:100E200091F018C090F017C0A9F016C0A8F000010A
:100E300001D0209A33D020AA30D090C018F091C0B1
:100E400019F0A8C016F0A9C017F0D7CF07F0D6CF79
:100E500006F01650065C17500758185008581950DD
:100E600009581AE31A8A48C000F049C001F000503E
:100E70000624166E01500720176E000E0820186E0B
:100E8000000E0920196E19C061F018C060F017C07B
:100E900079F016C078F08B8001D08B901AAC39D0E5
:100EA00062C018F063C019F07AC016F07BC017F06A
:100EB000D7CF07F0D6CF06F01650065C175007586C
:100EC000185008581950095823E3899A1A9C20ACE5
:100ED0001FD02E5202E12F521AE0D7CF07F0D6CF03
:100EE00006F02E500624166E2F500720176E000EA7
:100EF0000820186E000E0920196E19C093F018C052
:100F000092F017C0ABF016C0AAF0000101D0209CEF
:100F100033D020AC30D092C018F093C019F0AAC0E2
:100F200016F0ABC017F0D7CF07F0D6CF06F01650AB
:100F3000065C1750075818500858195009581AE3FA
:100F40001A8C4AC000F04BC001F000500624166E07
:100F500001500720176E000E0820186E000E0920A1
:100F6000196E19C063F018C062F017C07BF016C08C
:100F70007AF0898A01D0899A1AAE39D064C018F003
:100F800065C019F07CC016F07DC017F0D7CF07F010
:100F9000D6CF06F01650065C175007581850085860
:100FA0001950095823E389981A9E20AE1FD0305259
:100FB00002E131521AE0D7CF07F0D6CF06F0305019
:100FC0000624166E31500720176E000E0820186E8A
:100FD000000E0920196E19C095F018C094F017C0C2
:100FE000ADF016C0ACF0000101D0209E33D020AE91
:100FF00030D094C018F095C019F0ACC016F0ADC058
:1010000017F0D7CF07F0D6CF06F01650065C175072
:10101000075818500858195009581AE31A8E4CC02E
:1010200000F04DC001F000500624166E015007205C
:10103000176E000E0820186E000E0920196E19C0D8
:1010400065F018C064F017C07DF016C07CF0898888
:1010500001D089981BA039D066C018F067C019F07C
:101060007EC016F07FC017F0D7CF07F0D6CF06F0BE
:101070001650065C17500758185008581950095850
:1010800023E389961B9021A01FD0325202E13352F4
:101090001AE0D7CF07F0D6CF06F032500624166EEE
:1010A00033500720176E000E0820186E000E09201E
:1010B000196E19C097F018C096F017C0AFF016C09F
:1010C000AEF0000101D0219033D021A030D096C0E5
:1010D00018F097C019F0AEC016F0AFC017F0D7CF18
:1010E00007F0D6CF06F01650065C17500758185078
:1010F0000858195009581AE31B804EC000F04FC021
:1011000001F000500624166E01500720176E000EE5
:101110000820186E000E0920196E19C067F018C05B
:1011200066F017C07FF016C07EF0898601D08996E0
:101130001BA239D068C018F069C019F080C016F041
:1011400081C017F0D7CF07F0D6CF06F01650065C57
:1011500017500758185008581950095823E3899414
:101160001B9221A21FD0345202E135521AE0D7CF90
:1011700007F0D6CF06F034500624166E35500720FF
:10118000176E000E0820186E000E0920196E19C087
:1011900099F018C098F017C0B1F016C0B0F0000177
:1011A00001D0219233D021A230D098C018F099C03C
:1011B00019F0B0C016F0B1C017F0D7CF07F0D6CFF6
:1011C00006F01650065C175007581850085819506A
:1011D00009581AE31B8250C000F051C001F00050C2
:1011E0000624166E01500720176E000E0820186E98
:1011F000000E0920196E19C069F018C068F017C0F8
:1012000081F016C080F0898401D089941BA439D064
:101210006AC018F06BC019F082C016F083C017F0D6
:10122000D7CF07F0D6CF06F01650065C17500758F8
:10123000185008581950095823E389921B9421A487
:101240001FD0365202E137521AE0D7CF07F0D6CF7F
:1012500006F036500624166E37500720176E000E23
:101260000820186E000E0920196E19C09BF018C0D6
:101270009AF017C0B3F016C0B2F0000101D021946B
:1012800033D021A430D09AC018F09BC019F0B2C05E
:1012900016F0B3C017F0D7CF07F0D6CF06F0165030
:1012A000065C1750075818500858195009581AE387
:1012B0001B8452C000F053C001F000500624166E8B
:1012C00001500720176E000E0820186E000E09202E
:1012D000196E19C06BF018C06AF017C083F016C001
:1012E00082F0898201D089921BA639D06CC018F097
:1012F0006DC019F084C016F085C017F0D7CF07F085
:10130000D6CF06F01650065C1750075818500858EC
:101310001950095823E389901B9621A61FD03852F3
:1013200002E139521AE0D7CF07F0D6CF06F0385095
:101330000624166E39500720176E000E0820186E0E
:10134000000E0920196E19C09DF018C09CF017C03E
:10135000B5F016C0B4F0000101D0219633D021A61B
:1013600030D09CC018F09DC019F0B4C016F0B5C0C4
:1013700017F0D7CF07F0D6CF06F01650065C1750FF
:10138000075818500858195009581AE31B8654C0BA
:1013900000F055C001F000500624166E01500720E1
:1013A000176E000E0820186E000E0920196E19C065
:1013B0006DF018C06CF017C085F016C084F08980FD
:1013C00001D0899020501A24006E21501B20016EFC
:1013D00000100CE1010E095C09E3096A086A896AD8
:1013E0008B908B928B948B968B988B9AFCEF00F062
:1013F000330E115C11E112520CE000EEB6F0D89001
:101400001234E926000EEA22EECF22F0EFCF23F0CD
:1014100002D0236A226ADED0370E115C11E112522B
:101420000CE000EEB6F0D8901234E926000EEA2265
:10143000EECF24F0EFCF25F002D0256A246ACAD07F
:10144000390E115C03E0450E115C11E112520CE003
:1014500000EEB6F0D8901234E926000EEA22EECF64
:1014600026F0EFCF27F002D0276A266AB3D03C0ED1
:10147000115C11E112520CE000EEB6F0D89012347B
:10148000E926000EEA22EECF28F0EFCF29F002D0B5
:10149000296A286A9FD0410E115C11E112520CE0BA
:1014A00000EEB6F0D8901234E926000EEA22EECF14
:1014B0002AF0EFCF2BF002D02B6A2A6A8BD0430E92
:1014C000115C11E112520CE000EEB6F0D89012342B
:1014D000E926000EEA22EECF2CF0EFCF2DF002D05D
:1014E0002D6A2C6A77D0440E115C11E112520CE087
:1014F00000EEB6F0D8901234E926000EEA22EECFC4
:101500002EF0EFCF2FF002D02F6A2E6A63D0480E54
:10151000115C11E112520CE000EEB6F0D8901234DA
:10152000E926000EEA22EECF30F0EFCF31F002D004
:10153000316A306A4FD0550E115C11E112520CE045
:1015400000EEB6F0D8901234E926000EEA22EECF73
:1015500032F0EFCF33F002D0336A326A3BD0570E0D
:10156000115C11E112520CE000EEB6F0D89012348A
:10157000E926000EEA22EECF34F0EFCF35F002D0AC
:10158000356A346A27D0580E115C11E112520CE012
:1015900000EEB6F0D8901234E926000EEA22EECF23
:1015A00036F0EFCF37F002D0376A366A13D0590ED3
:1015B000115C10E112520CE000EEB6F0D89012343B
:1015C000E926000EEA22EECF38F0EFCF39F002D054
:1015D000396A386A11681200420E135C0AE114522B
:1015E00004E11CD88A941C6A03D08A8414C01CF0BD
:1015F00013D07B0E135C10E11B6A1A6A216A206A01
:1016000089908992899489968998899A8B908B92EE
:101610008B948B968B988B9A136812001B6A1A6AAC
:10162000216A206A89908992899489968998899AF1
:101630008B908B928B948B968B988B9A236A226AD1
:10164000256A246A276A266A296A286A2B6A2A6A0E
:101650002D6A2C6A2F6A2E6A316A306A336A326ABE
:10166000356A346A376A366A396A386A120060EC59
:1016700000F00A6EBE0E0A5C04E3FE0E0A5C01E294
:101680000C6A0AAE09D00C6ABD0E0A5C04E10AC0FD
:101690000CF0136814680FD0BD0E0C5C0CE113281D
:1016A00003E10AC013F007D00AC014F0145203E09B
:1016B0008A84FCEF00F0DBD7A20EB96FC30EB86FBF
:1016C000980EBB6F990EBA6F930EBD6FC20EBC6FB2
:1016D0008F0EBF6F120EBE6F8A0EC16F880EC06F65
:1016E000860EC36F230EC26F810EC56FE10EC46FED
:1016F0007D0EC76FC30EC66F790EC96FC50EC86F5A
:10170000750ECB6FE80ECA6F720ECD6F2B0ECC6FBD
:101710006E0ECF6F8B0ECE6F6B0ED16F0A0ED06F29
:10172000670ED36FA40ED26F640ED56F5B0ED46FAD
:10173000610ED76F2C0ED66F5E0ED96F160ED86F56
:101740005B0EDB6F1A0EDA6F580EDD6F360EDC6F34
:10175000550EDF6F6A0EDE6F520EE16FB40EE06F52
:10176000500EE36F150EE26F4D0EE56F8A0EE46FBB
:101770004B0EE76F140EE66F480EE96FB30EE86F7D
:10178000460EEB6F640EEA6F440EED6F290EEC6FA0
:10179000410EEF6FEE693F0EF16FE70EF06F3D0EF9
:1017A000F36FE00EF26F3B0EF56FEA0EF46F3A0E38
:1017B000F76F030EF66F380EF96F2C0EF86F360EBA
:1017C000FB6F640EFA6F340EFD6FAA0EFC6F320EC3
:1017D000FF6FFE0EFE6F310E0101016F600E006F94
:1017E0002F0E036FCF0E026F2E0E056F4B0E046F80
:1017F0002C0E076FD30E066F2B0E096F670E086F46
:101800002A0E0B6F060E0A6F280E0D6FB10E0C6FAD
:10181000270E0F6F660E0E6F260E116F106F240EBF
:10182000136FF10E126F230E156FC50E146F220E7B
:10183000176FA20E166F210E196F890E186F200EEA
:101840001B6F790E1A6F1F0E1D6F710E1C6F1E0E0F
:101850001F6F710E1E6F1D0E216F7A0E206F1C0EF2
:10186000236F8B0E226F1B0E256FA30E246F1A0E93
:10187000276FC30E266F190E296FE90E286F190EF8
:101880002B6F170E2A6F180E2D6F4B0E2C6F170E25
:101890002F6F860E2E6F160E316FC70E306F160E1D
:1018A000336F0E0E326F150E356F5B0E346F140EE4
:1018B000376FAD0E366F140E396F050E386F130E7D
:1018C0003B6F630E3A6F120E3D6FC50E3C6F120EEA
:1018D0003F6F2D0E3E6F110E416F990E406F110E2E
:1018E000436F0A0E426F100E456F800E446F0F0E4D
:1018F000476FFA0E466F0F0E496F780E486F0E0E47
:101900004B6FFA0E4A6F0E0E4D6F810E4C6F0E0E1E
:101910004F6F0B0E4E6F0D0E516F990E506F0D0ED7
:10192000536F2B0E526F0C0E556FC00E546F0C0E72
:10193000576F580E566F0B0E596FF40E586F0B0EF3
:101940005B6F930E5A6F0B0E5D6F350E5C6F0A0E58
:101950005F6FDA0E5E6F0A0E616F820E606F0A0EA5
:10196000636F2C0E626F090E656FDA0E646F090EDD
:10197000676F8A0E666F090E696F3C0E686F080EFE
:101980006B6FF10E6A6F080E6D6FA90E6C6F080E0B
:101990006F6F620E6E6F080E716F1E0E706F070E06
:1019A000736FDC0E726F070E756F9C0E746F070EEF
:1019B000776F5F0E766F070E796F230E786F060EC6
:1019C0007B6FE90E7A6F060E7D6FB10E7C6F060E8F
:1019D0007F6F7A0E7E6F060E816F460E806F060E49
:1019E000836F130E826F050E856FE10E846F050EF7
:1019F000876FB20E866F050E896F830E886F050E96
:101A00008B6F570E8A6F050E8D6F2B0E8C6F050E28
:101A10008F6F010E8E6F040E916FD90E906F040EB2
:101A2000936FB10E926F040E956F8B0E946F040E30
:101A3000976F660E966F040E996F430E986F040EA3
:101A40009B6F200E9A6F030E9D6FFE0E9C6F030E10
:101A50009F6FDE0E9E6F030EA16FBF0EA06F030E71
:101A6000A36FA00EA26F030EA56F830EA46F030ECB
:101A7000A76F660EA66F030EA96F4B0EA86F030E1D
:101A8000AB6F300EAA6F030EAD6F160EAC6F020E69
:101A9000AF6FFD0EAE6F020EB16FE50EB06F020EAE
:101AA000B36FCD0EB26F020EB56FB60EB46F0001FC
:101AB00012000401B96B8C0EB86FBB6B8E0EBA6F3F
:101AC000BD6B900EBC6FBF6B910EBE6FC16B930E62
:101AD000C06FC36B950EC26FC56B960EC46FC76B9C
:101AE000980EC66FC96B9A0EC86FCB6B9C0ECA6FEF
:101AF000CD6B9D0ECC6FCF6B9F0ECE6FD16BA10EB9
:101B0000D06FD36BA20ED26FD56BA40ED46FD76BF0
:101B1000A60ED66FD96BA80ED86FDB6BA90EDA6F45
:101B2000DD6BAB0EDC6FDF6BAD0EDE6FE16BAE0E0F
:101B3000E06FE36BB00EE26FE56BB20EE46FE76B44
:101B4000B30EE66FE96BB50EE86FEB6BB70EEA6F9D
:101B5000ED6BB90EEC6FEF6BBA0EEE6FF16BBC0E66
:101B6000F06FF36BBE0EF26FF56BBF0EF46FF76B99
:101B7000C10EF66FF96BC30EF86FFB6BC40EFA6FF4
:101B8000FD6BC60EFC6FFF6BC80EFE6F0501016B8F
:101B9000CA0E006F036BCB0E026F056BCD0E046F88
:101BA000076BCF0E066F096BD00E086F0B6BD20E52
:101BB0000A6F0D6BD40E0C6F0F6BD50E0E6F116B81
:101BC000D70E106F136BD90E126F156BDB0E146FDF
:101BD000176BDC0E166F196BDE0E186F1B6BE00EA9
:101BE0001A6F1D6BE10E1C6F1F6BE30E1E6F216BD6
:101BF000E50E206F236BE60E226F256BE80E246F37
:101C0000276BEA0E266F296BEC0E286F2B6BED0EFF
:101C10002A6F2D6BEF0E2C6F2F6BF10E2E6F316B29
:101C2000F20E306F336BF40E326F356BF60E346F8D
:101C3000376BF80E366F396BF90E386F3B6BFB0E56
:101C40003A6F3D6BFD0E3C6F3F6BFE0E3E6F010E1B
:101C5000416F406B436F020E426F010E456F030EE2
:101C6000446F010E476F050E466F010E496F070E58
:101C7000486F010E4B6F090E4A6F010E4D6F0A0E31
:101C80004C6F010E4F6F0C0E4E6F010E516F0E0E0A
:101C9000506F010E536F0F0E526F010E556F110EE4
:101CA000546F010E576F130E566F010E596F140EBD
:101CB000586F010E5B6F160E5A6F010E5D6F180E96
:101CC0005C6F010E5F6F1A0E5E6F010E616F1B0E6F
:101CD000606F010E636F1D0E626F010E656F1F0E48
:101CE000646F010E676F200E666F010E696F220E22
:101CF000686F010E6B6F240E6A6F010E6D6F250EFB
:101D00006C6F010E6F6F270E6E6F010E716F290ED3
:101D1000706F010E736F2B0E726F010E756F2C0EAC
:101D2000746F010E776F2E0E766F010E796F300E85
:101D3000786F010E7B6F310E7A6F010E7D6F330E5F
:101D40007C6F010E7F6F350E7E6F010E816F360E38
:101D5000806F010E836F380E826F010E856F3A0E11
:101D6000846F010E876F3C0E866F010E896F3D0EEA
:101D7000886F010E8B6F3F0E8A6F010E8D6F410EC3
:101D80008C6F010E8F6F420E8E6F010E916F440E9D
:101D9000906F010E936F460E926F010E956F480E75
:101DA000946F010E976F490E966F010E996F4B0E4F
:101DB000986F010E9B6F4D0E9A6F010E9D6F4E0E28
:101DC0009C6F010E9F6F500E9E6F010EA16F520E01
:101DD000A06F010EA36F530EA26F010EA56F550EDB
:101DE000A46F010EA76F570EA66F010EA96F590EB3
:101DF000A86F010EAB6F5A0EAA6F010EAD6F5C0E8D
:101E0000AC6F010EAF6F5E0EAE6F010EB16F5F0E65
:101E1000B06F010EB36F610EB26F010EB56F630E3E
:101E2000B46FB96BEF0EB86FBB6BF20EBA6FBD6BD0
:101E3000F50EBC6FBF6BF90EBE6FC16BFC0EC06FB1
:101E4000C36BC269010EC56F030EC46F010EC76F6D
:101E5000060EC66F010EC96F090EC86F010ECB6F5B
:101E60000D0ECA6F010ECD6F100ECC6F010ECF6F2D
:101E7000140ECE6F010ED16F170ED06F010ED36FFF
:101E80001A0ED26F010ED56F1E0ED46F010ED76FD2
:101E9000210ED66F010ED96F240ED86F010EDB6FA5
:101EA000280EDA6F010EDD6F2B0EDC6F010EDF6F77
:101EB0002E0EDE6F010EE16F320EE06F010EE36F4A
:101EC000350EE26F010EE56F390EE46F010EE76F1C
:101ED0003C0EE66F010EE96F3F0EE86F010EEB6FEF
:101EE000430EEA6F010EED6F460EEC6F010EEF6FC1
:101EF000490EEE6F010EF16F4D0EF06F010EF36F94
:101F0000500EF26F010EF56F540EF46F010EF76F65
:101F1000570EF66F010EF96F5A0EF86F010EFB6F38
:101F20005E0EFA6F010EFD6F610EFC6F010EFF6F0A
:101F3000640EFE6F010E0601016F680E006F010E48
:101F4000036F6B0E026F010E056F6E0E046F010EB4
:101F5000076F720E066F010E096F750E086F010E86
:101F60000B6F790E0A6F010E0D6F7C0E0C6F010E58
:101F70000F6F7F0E0E6F010E116F830E106F010E2B
:101F8000136F860E126F010E156F890E146F010EFE
:101F9000176F8D0E166F010E196F900E186F010ED0
:101FA0001B6F930E1A6F010E1D6F970E1C6F010EA3
:101FB0001F6F9A0E1E6F010E216F9E0E206F010E75
:101FC000236FA10E226F010E256FA40E246F010E48
:101FD000276FA80E266F010E296FAB0E286F010E1A
:101FE0002B6FAE0E2A6F010E2D6FB20E2C6F010EED
:101FF0002F6FB50E2E6F010E316FB80E306F010EC0
:10200000336FBC0E326F010E356FBF0E346F010E91
:10201000376FC30E366F010E396FC60E386F010E63
:102020003B6FC90E3A6F010E3D6FCD0E3C6F010E36
:102030003F6FD00E3E6F010E416FD30E406F010E09
:10204000436FD70E426F010E456FDA0E446F010EDB
:10205000476FDE0E466F010E496FE10E486F010EAD
:102060004B6FE40E4A6F010E4D6FE80E4C6F010E80
:102070004F6FEB0E4E6F010E516FEE0E506F010E53
:10208000536FF20E526F010E556FF50E546F010E25
:10209000576FF80E566F010E596FFC0E586F010EF8
:1020A0005B6F5A69020E5D6F030E5C6F020E5F6F0D
:1020B000060E5E6F020E616F090E606F020E636F97
:1020C0000D0E626F020E656F100E646F020E676F69
:1020D000130E666F020E696F170E686F020E6B6F3C
:1020E0001A0E6A6F020E6D6F1D0E6C6F020E6F6F0F
:1020F000210E6E6F020E716F240E706F020E736FE1
:10210000280E726F020E756F2B0E746F020E776FB2
:102110002E0E766F020E796F320E786F020E7B6F85
:10212000350E7A6F020E7D6F380E7C6F020E7F6F58
:102130003C0E7E6F020E816F3F0E806F020E836F2A
:10214000420E826F020E856F460E846F020E876FFD
:10215000490E866F020E896F4D0E886F020E8B6FCF
:10216000500E8A6F020E8D6F530E8C6F020E8F6FA2
:10217000570E8E6F020E916F5A0E906F020E936F74
:102180005D0E926F020E956F610E946F020E976F47
:10219000640E966F020E996F680E986F020E9B6F19
:1021A0006B0E9A6F020E9D6F6E0E9C6F020E9F6FEC
:1021B000720E9E6F020EA16F750EA06F020EA36FBE
:1021C000780EA26F020EA56F7C0EA46F020EA76F91
:1021D0007F0EA66F020EA96F820EA86F020EAB6F64
:1021E000860EAA6F020EAD6F890EAC6F020EAF6F36
:1021F0008D0EAE6F020EB16F900EB06F020EB36F08
:10220000930EB26F020EB56F970EB46FB96B910E4D
:10221000B86FBB6B950EBA6FBD6B990EBC6FBF6B81
:102220009D0EBE6FC16BA20EC06FC36BA60EC26FB8
:10223000C56BAA0EC46FC76BAE0EC66FC96BB20E6C
:10224000C86FCB6BB60ECA6FCD6BBA0ECC6FCF6BAF
:10225000BE0ECE6FD16BC20ED06FD36BC60ED26FD7
:10226000D56BCB0ED46FD76BCF0ED66FD96BD30E89
:10227000D86FDB6BD70EDA6FDD6BDB0EDC6FDF6BDD
:10228000DF0EDE6FE16BE30EE06FE36BE70EE26FF4
:10229000E56BEB0EE46FE76BF00EE66FE96BF40EA7
:1022A000E86FEB6BF80EEA6FED6BFC0EEC6F010E56
:1022B000EF6FEE6BF16F040EF06F010EF36F080E0F
:1022C000F26F010EF56F0C0EF46F010EF76F100E2A
:1022D000F66F010EF96F140EF86F010EFB6F190EF9
:1022E000FA6F010EFD6F1D0EFC6F010EFF6F210EC8
:1022F000FE6F010E0701016F250E006F010E036FC7
:10230000290E026F010E056F2D0E046F010E076F6F
:10231000310E066F010E096F350E086F010E0B6F3F
:10232000390E0A6F010E0D6F3D0E0C6F010E0F6F0F
:10233000420E0E6F010E116F460E106F010E136FDD
:102340004A0E126F010E156F4E0E146F010E176FAD
:10235000520E166F010E196F560E186F010E1B6F7D
:102360005A0E1A6F010E1D6F5E0E1C6F010E1F6F4D
:10237000620E1E6F010E216F660E206F010E236F1D
:102380006B0E226F010E256F6F0E246F010E276FEB
:10239000730E266F010E296F770E286F010E2B6FBB
:1023A0007B0E2A6F010E2D6F7F0E2C6F010E2F6F8B
:1023B000830E2E6F010E316F870E306F010E336F5B
:1023C0008B0E326F010E356F8F0E346F010E376F2B
:1023D000940E366F010E396F980E386F010E3B6FF9
:1023E0009C0E3A6F010E3D6FA00E3C6F010E3F6FC9
:1023F000A40E3E6F010E416FA80E406F010E436F99
:10240000AC0E426F010E456FB00E446F010E476F68
:10241000B40E466F010E496FB80E486F010E4B6F38
:10242000BD0E4A6F010E4D6FC10E4C6F010E4F6F06
:10243000C50E4E6F010E516FC90E506F010E536FD6
:10244000CD0E526F010E556FD10E546F010E576FA6
:10245000D50E566F010E596FD90E586F010E5B6F76
:10246000DD0E5A6F010E5D6FE10E5C6F010E5F6F46
:10247000E60E5E6F010E616FEA0E606F010E636F14
:10248000EE0E626F010E656FF20E646F010E676FE4
:10249000F60E666F010E696FFA0E686F010E6B6FB4
:1024A000FE0E6A6F020E6D6F6C6F6F6F060E6E6FB1
:1024B000020E716F0A0E706F020E736F0F0E726F45
:1024C000020E756F130E746F020E776F170E766F14
:1024D000020E796F1B0E786F020E7B6F1F0E7A6FE4
:1024E000020E7D6F230E7C6F020E7F6F270E7E6FB4
:1024F000020E816F2B0E806F020E836F2F0E826F84
:10250000020E856F330E846F020E876F380E866F52
:10251000020E896F3C0E886F020E8B6F400E8A6F21
:10252000020E8D6F440E8C6F020E8F6F480E8E6FF1
:10253000020E916F4C0E906F020E936F500E926FC1
:10254000020E956F540E946F020E976F580E966F91
:10255000020E996F5C0E986F020E9B6F610E9A6F60
:10256000020E9D6F650E9C6F020E9F6F690E9E6F2F
:10257000020EA16F6D0EA06F020EA36F710EA26FFF
:10258000020EA56F750EA46F020EA76F790EA66FCF
:10259000020EA96F7D0EA86F020EAB6F810EAA6F9F
:1025A000020EAD6F850EAC6F020EAF6F8A0EAE6F6E
:1025B000020EB16F8E0EB06F020EB36F920EB26F3D
:1025C000020EB56F960EB46FB96B820EB86FBB6B0F
:1025D000840EBA6FBD6B860EBC6FBF6B880EBE6F6C
:1025E000C16B8A0EC06FC36B8B0EC26FC56B8D0E35
:1025F000C46FC76B8F0EC66FC96B910EC86FCB6B64
:10260000920ECA6FCD6B940ECC6FCF6B960ECE6FC1
:10261000D16B980ED06FD36B9A0ED26FD56B9B0E89
:10262000D46FD76B9D0ED66FD96B9F0ED86FDB6BB7
:10263000A10EDA6FDD6BA20EDC6FDF6BA40EDE6F16
:10264000E16BA60EE06FE36BA80EE26FE56BAA0EDE
:10265000E46FE76BAB0EE66FE96BAD0EE86FEB6B0B
:10266000AF0EEA6FED6BB10EEC6FEF6BB20EEE6F6B
:10267000F16BB40EF06FF36BB60EF26FF56BB80E34
:10268000F46FF76BBA0EF66FF96BBB0EF86FFB6B5E
:10269000BD0EFA6FFD6BBF0EFC6FFF6BC10EFE6FC0
:1026A0000801016BC30E006F036BC40E026F056B54
:1026B000C60E046F076BC80E066F096BCA0E086F53
:1026C0000B6BCB0E0A6F0D6BCD0E0C6F0F6BCF0E1D
:1026D0000E6F116BD10E106F136BD30E126F156B43
:1026E000D40E146F176BD60E166F196BD80E186FA9
:1026F0001B6BDA0E1A6F1D6BDB0E1C6F1F6BDD0E72
:102700001E6F216BDF0E206F236BE10E226F256B96
:10271000E30E246F276BE40E266F296BE60E286FFD
:102720002B6BE80E2A6F2D6BEA0E2C6F2F6BEB0EC6
:102730002E6F316BED0E306F336BEF0E326F356BEA
:10274000F10E346F376BF30E366F396BF40E386F52
:102750003B6BF60E3A6F3D6BF80E3C6F3F6BFA0E1B
:102760003E6F416BFB0E406F436BFD0E426F456B3E
:102770004469010E476F466F496F030E486F010EA3
:102780004B6F040E4A6F010E4D6F060E4C6F010E1B
:102790004F6F080E4E6F010E516F0A0E506F010EF3
:1027A000536F0B0E526F010E556F0D0E546F010ECD
:1027B000576F0F0E566F010E596F110E586F010EA5
:1027C0005B6F130E5A6F010E5D6F140E5C6F010E7E
:1027D0005F6F160E5E6F010E616F180E606F010E57
:1027E000636F1A0E626F010E656F1B0E646F010E30
:1027F000676F1D0E666F010E696F1F0E686F010E09
:102800006B6F210E6A6F010E6D6F230E6C6F010EE0
:102810006F6F240E6E6F010E716F260E706F010EBA
:10282000736F280E726F010E756F2A0E746F010E92
:10283000776F2C0E766F010E796F2D0E786F010E6B
:102840007B6F2F0E7A6F010E7D6F310E7C6F010E44
:102850007F6F330E7E6F010E816F340E806F010E1D
:10286000836F360E826F010E856F380E846F010EF6
:10287000876F3A0E866F010E896F3C0E886F010ECE
:102880008B6F3D0E8A6F010E8D6F3F0E8C6F010EA8
:102890008F6F410E8E6F010E916F430E906F010E80
:1028A000936F440E926F010E956F460E946F010E5A
:1028B000976F480E966F010E996F4A0E986F010E32
:1028C0009B6F4C0E9A6F010E9D6F4D0E9C6F010E0B
:1028D0009F6F4F0E9E6F010EA16F510EA06F010EE4
:1028E000A36F530EA26F010EA56F540EA46F010EBD
:1028F000A76F560EA66F010EA96F580EA86F010E96
:10290000AB6F5A0EAA6F010EAD6F5C0EAC6F010E6D
:10291000AF6F5D0EAE6F010EB16F5F0EB06F010E47
:10292000B36F610EB26F010EB56F630EB46F03012A
:10293000B96B3E0EB86FBB6B3F0EBA6FBD6B400EEE
:10294000BC6FBF6B410EBE6FC16B430EC06FC36BDC
:10295000440EC26FC56B450EC46FC76B460EC66F83
:10296000C96B480EC86FCB6B490ECA6FCD6B4A0E50
:10297000CC6FCF6B4B0ECE6FD16B4D0ED06FD36B38
:102980004E0ED26FD56B4F0ED46FD76B500ED66FE5
:10299000D96B510ED86FDB6B530EDA6FDD6B540EB3
:1029A000DC6FDF6B550EDE6FE16B560EE06FE36B95
:1029B000580EE26FE56B590EE46FE76B5A0EE66F47
:1029C000E96B5B0EE86FEB6B5D0EEA6FED6B5E0E15
:1029D000EC6FEF6B5F0EEE6FF16B600EF06FF36BF1
:1029E000620EF26FF56B630EF46FF76B640EF66FA9
:1029F000F96B650EF86FFB6B670EFA6FFD6B680E77
:102A0000FC6FFF6B690EFE6F0401016B6A0E006FB5
:102A1000036B6B0E026F056B6D0E046F076B6E0E12
:102A2000066F096B6F0E086F0B6B700E0A6F0D6BE4
:102A3000720E0C6F0F6B730E0E6F116B740E106FA6
:102A4000136B750E126F156B770E146F176B780E74
:102A5000166F196B790E186F1B6B7A0E1A6F1D6B40
:102A60007C0E1C6F1F6B7D0E1E6F216B7E0E206F08
:102A7000236B7F0E226F256B810E246F276B820ED6
:102A8000266F296B830E286F2B6B840E2A6F2D6B9C
:102A9000850E2C6F2F6B870E2E6F316B880E306F6B
:102AA000336B890E326F356B8A0E346F376B8C0E39
:102AB000366F396B8D0E386F3B6B8E0E3A6F3D6BF8
:102AC0008F0E3C6F3F6B910E3E6F416B920E406FCD
:102AD000436B930E426F456B940E446F476B960E9B
:102AE000466F496B970E486F4B6B980E4A6F4D6B54
:102AF000990E4C6F4F6B9B0E4E6F516B9C0E506F2F
:102B0000536B9D0E526F556B9E0E546F576B9F0EFD
:102B1000566F596BA10E586F5B6BA20E5A6F5D6BAF
:102B2000A30E5C6F5F6BA40E5E6F616BA60E606F91
:102B3000636BA70E626F656BA80E646F676BA90E5F
:102B4000666F696BAB0E686F6B6BAC0E6A6F6D6B0B
:102B5000AD0E6C6F6F6BAE0E6E6F716BB00E706FF3
:102B6000736BB10E726F756BB20E746F776BB30EC1
:102B7000766F796BB50E786F7B6BB60E7A6F7D6B67
:102B8000B70E7C6F7F6BB80E7E6F816BB90E806F56
:102B9000836BBB0E826F856BBC0E846F876BBD0E23
:102BA000866F896BBE0E886F8B6BC00E8A6F8D6BC4
:102BB000C10E8C6F8F6BC20E8E6F916BC30E906FB8
:102BC000936BC50E926F956BC60E946F976BC70E85
:102BD000966F996BC80E986F9B6BCA0E9A6F9D6B20
:102BE000CB0E9C6F9F6BCC0E9E6FA16BCD0EA06F1A
:102BF000A36BCF0EA26FA56BD00EA46FA76BD10EE7
:102C0000A66FA96BD20EA86FAB6BD30EAA6FAD6B7C
:102C1000D50EAC6FAF6BD60EAE6FB16BD70EB06F7B
:102C2000B36BD80EB26FB56BDA0EB46F0801B96B27
:102C3000740EB86FBB6B750EBA6FBD6BBC6FBF6B9C
:102C4000760EBE6FC16B770EC06FC36B780EC26F0E
:102C5000C56B790EC46FC76BC66FC96B7A0EC86F30
:102C6000CB6B7B0ECA6FCD6B7C0ECC6FCF6B7D0EAA
:102C7000CE6FD16BD06FD36B7E0ED26FD56B7F0EC4
:102C8000D46FD76B800ED66FD96B810ED86FDB6B8C
:102C9000820EDA6FDD6BDC6FDF6B830EDE6FE16B54
:102CA000840EE06FE36B850EE26FE56B860EE46FDA
:102CB000E76BE66FE96B870EE86FEB6B880EEA6FE8
:102CC000ED6B890EEC6FEF6B8A0EEE6FF16BF06FB0
:102CD000F36B8B0EF26FF56B8C0EF46FF76B8D0E42
:102CE000F66FF96B8E0EF86FFB6B8F0EFA6FFD6B44
:102CF000FC6FFF6B900EFE6F0901016B910E006F70
:102D0000036B920E026F056B930E046F076B066FD9
:102D1000096B940E086F0B6B950E0A6F0D6B960E78
:102D20000C6F0F6B970E0E6F116B106F136B980E6D
:102D3000126F156B990E146F176B9A0E166F196B35
:102D40009B0E186F1B6B9C0E1A6F1D6B1C6F1F6BFD
:102D50009D0E1E6F216B9E0E206F236B9F0E226FA8
:102D6000256BA00E246F276B266F296BA10E286F91
:102D70002B6BA20E2A6F2D6BA30E2C6F2F6BA40E44
:102D80002E6F316B306F336BA50E326F356BA60E25
:102D9000346F376BA70E366F396BA80E386F3B6BED
:102DA000A90E3A6F3D6B3C6F3F6BAA0E3E6F416BB5
:102DB000AB0E406F436BAC0E426F456BAD0E446F74
:102DC000476B466F496BAE0E486F4B6BAF0E4A6F49
:102DD0004D6BB00E4C6F4F6BB10E4E6F516B506F11
:102DE000536BB20E526F556BB30E546F576BB40EDC
:102DF000566F596BB50E586F5B6BB60E5A6F5D6BA5
:102E00005C6F5F6BB70E5E6F616BB80E606F636B6C
:102E1000B90E626F656BBA0E646F676B666F696B34
:102E2000BB0E686F6B6BBC0E6A6F6D6BBD0E6C6F0B
:102E30006F6BBE0E6E6F716B706F736BBF0E726FC8
:102E4000756BC00E746F776BC10E766F796BC20EA7
:102E5000786F7B6BC30E7A6F7D6B7C6F7F6BC40E5C
:102E60007E6F816BC50E806F836BC60E826F856B24
:102E7000C70E846F876B866F896BC80E886F8B6BEC
:102E8000C90E8A6F8D6BCA0E8C6F8F6BCB0E8E6FD7
:102E9000916B906F936BCC0E926F956BCD0E946F80
:102EA000976BCE0E966F996BCF0E986F9B6BD00E73
:102EB0009A6F9D6B9C6F9F6BD10E9E6FA16BD20E14
:102EC000A06FA36BD30EA26FA56BD40EA46FA76BDC
:102ED000A66FA96BD50EA86FAB6BD60EAA6FAD6BA4
:102EE000D70EAC6FAF6BD80EAE6FB16BB06FB36B6C
:102EF000D90EB26FB56BDA0EB46F0101B96B7E0EED
:102F0000B86FBB6B820EBA6FBD6B860EBC6FBF6BAA
:102F10008A0EBE6FC16B8F0EC06FC36B930EC26FF4
:102F2000C56B970EC46FC76B9B0EC66FC96BA00EA7
:102F3000C86FCB6BA40ECA6FCD6BA80ECC6FCF6BD6
:102F4000AC0ECE6FD16BB10ED06FD36BB50ED26F0E
:102F5000D56BB90ED46FD76BBD0ED66FD96BC20EC1
:102F6000D86FDB6BC60EDA6FDD6BCA0EDC6FDF6B02
:102F7000CE0EDE6FE16BD30EE06FE36BD70EE26F28
:102F8000E56BDB0EE46FE76BDF0EE66FE96BE40EDB
:102F9000E86FEB6BE80EEA6FED6BEC0EEC6FEF6B2E
:102FA000F00EEE6FF16BF50EF06FF36BF90EF26F42
:102FB000F56BFD0EF46F010EF76FF66FF96F060EED
:102FC000F86F010EFB6F0A0EFA6F010EFD6F0E0E09
:102FD000FC6F010EFF6F120EFE6F010E0201016FFA
:102FE000170E006F010E036F1B0E026F010E056FAF
:102FF0001F0E046F010E076F230E066F010E096F7F
:10300000280E086F010E0B6F2C0E0A6F010E0D6F4C
:10301000300E0C6F010E0F6F350E0E6F010E116F1B
:10302000390E106F010E136F3D0E126F010E156FEA
:10303000410E146F010E176F460E166F010E196FB9
:103040004A0E186F010E1B6F4E0E1A6F010E1D6F88
:10305000520E1C6F010E1F6F570E1E6F010E216F57
:103060005B0E206F010E236F5F0E226F010E256F26
:10307000630E246F010E276F680E266F010E296FF5
:103080006C0E286F010E2B6F700E2A6F010E2D6FC4
:10309000740E2C6F010E2F6F790E2E6F010E316F93
:1030A0007D0E306F010E336F810E326F010E356F62
:1030B000850E346F010E376F8A0E366F010E396F31
:1030C0008E0E386F010E3B6F920E3A6F010E3D6F00
:1030D000960E3C6F010E3F6F9B0E3E6F010E416FCF
:1030E0009F0E406F010E436FA30E426F010E456F9E
:1030F000A70E446F010E476FAC0E466F010E496F6D
:10310000B00E486F010E4B6FB40E4A6F010E4D6F3B
:10311000B80E4C6F010E4F6FBD0E4E6F010E516F0A
:10312000C10E506F010E536FC50E526F010E556FD9
:10313000C90E546F010E576FCE0E566F010E596FA8
:10314000D20E586F010E5B6FD60E5A6F010E5D6F77
:10315000DA0E5C6F010E5F6FDF0E5E6F010E616F46
:10316000E30E606F010E636FE70E626F010E656F15
:10317000EC0E646F010E676FF00E666F010E696FE3
:10318000F40E686F010E6B6FF80E6A6F010E6D6FB3
:10319000FD0E6C6F020E6F6F010E6E6F020E716F7F
:1031A000050E706F020E736F090E726F020E756F4F
:1031B0000E0E746F020E776F120E766F020E796F1D
:1031C000160E786F020E7B6F1A0E7A6F020E7D6FED
:1031D0001F0E7C6F020E7F6F230E7E6F020E816FBB
:1031E000270E806F020E836F2B0E826F020E856F8B
:1031F000300E846F020E876F340E866F020E896F59
:10320000380E886F020E8B6F3C0E8A6F020E8D6F28
:10321000410E8C6F020E8F6F450E8E6F020E916FF6
:10322000490E906F020E936F4D0E926F020E956FC6
:10323000520E946F020E976F560E966F020E996F94
:103240005A0E986F020E9B6F5E0E9A6F020E9D6F64
:10325000630E9C6F020E9F6F670E9E6F020EA16F32
:103260006B0EA06F020EA36F6F0EA26F020EA56F02
:10327000740EA46F020EA76F780EA66F020EA96FD0
:103280007C0EA86F020EAB6F800EAA6F020EAD6FA0
:10329000850EAC6F020EAF6F890EAE6F020EB16F6E
:1032A0008D0EB06F020EB36F910EB26F020EB56F3E
:1032B000960EB46F0901B96B650EB86FBB6B660EE5
:1032C000BA6FBD6BBC6FBF6B670EBE6FC16BC06F5B
:1032D000C36B680EC26FC56B690EC46FC76BC66FD8
:1032E000C96B6A0EC86FCB6B6B0ECA6FCD6BCC6FA0
:1032F000CF6B6C0ECE6FD16BD06FD36B6D0ED26F68
:10330000D56B6E0ED46FD76BD66FD96B6F0ED86F2F
:10331000DB6BDA6FDD6B700EDC6FDF6B710EDE6FF7
:10332000E16BE06FE36B720EE26FE56B730EE46FBF
:10333000E76BE66FE96B740EE86FEB6BEA6FED6BB2
:10334000750EEC6FEF6B760EEE6FF16BF06FF36B4B
:10335000770EF26FF56B780EF46FF76BF66FF96B13
:10336000790EF86FFB6BFA6FFD6B7A0EFC6FFF6BDB
:103370007B0EFE6F0A01016B006F036B7C0E026F08
:10338000056B046F076B7D0E066F096B7E0E086F71
:103390000B6B0A6F0D6B7F0E0C6F0F6B800E0E6F39
:1033A000116B106F136B810E126F156B146F176B0F
:1033B000820E166F196B830E186F1B6B1A6F1D6BC5
:1033C000840E1C6F1F6B850E1E6F216B206F236B8D
:1033D000860E226F256B246F276B870E266F296B55
:1033E000880E286F2B6B2A6F2D6B890E2C6F2F6B1D
:1033F0002E6F316B8A0E306F336B8B0E326F356BE5
:10340000346F376B8C0E366F396B8D0E386F3B6BAC
:103410003A6F3D6B8E0E3C6F3F6B3E6F416B8F0E74
:10342000406F436B900E426F456B446F476B910E3C
:10343000466F496B920E486F4B6B4A6F4D6B930E04
:103440004C6F4F6B4E6F516B940E506F536B950ECC
:10345000526F556B546F576B960E566F596B586F72
:103460005B6B970E5A6F5D6B980E5C6F5F6B5E6F58
:10347000616B990E606F636B9A0E626F656B646F20
:10348000676B9B0E666F696B686F6B6B9C0E6A6FE8
:103490006D6B9D0E6C6F6F6B6E6F716B9E0E706FB0
:1034A000736B9F0E726F756B746F776BA00E766F78
:1034B000796B786F7B6BA10E7A6F7D6BA20E7C6F40
:1034C0007F6B7E6F816BA30E806F836B826F856BCA
:1034D000A40E846F876BA50E866F896B886F8B6BCC
:1034E000A60E8A6F8D6BA70E8C6F8F6B8E6F916B94
:1034F000A80E906F936B926F956BA90E946F976B5C
:10350000AA0E966F996B986F9B6BAB0E9A6F9D6B23
:10351000AC0E9C6F9F6B9E6FA16BAD0EA06FA36BEB
:10352000A26FA56BAE0EA46FA76BAF0EA66FA96BB3
:10353000A86FAB6BB00EAA6FAD6BAC6FAF6BB10E7B
:10354000AE6FB16BB20EB06FB36BB26FB56BB30E43
:10355000B46FB96B8C0EB86FBB6B8D0EBA6FBD6B51
:103560008E0EBC6FBF6B8F0EBE6FC16BC06FC36B17
:10357000900EC26FC56B910EC46FC76B920EC66F73
:10358000C96BC86FCB6B930ECA6FCD6B940ECC6FAB
:10359000CF6B950ECE6FD16B960ED06FD36BD26F73
:1035A000D56B970ED46FD76B980ED66FD96B990EDB
:1035B000D86FDB6BDA6FDD6B9A0EDC6FDF6B9B0E07
:1035C000DE6FE16B9C0EE06FE36B9D0EE26FE56BCF
:1035D000E46FE76B9E0EE66FE96B9F0EE86FEB6B97
:1035E000A00EEA6FED6BEC6FEF6BA10EEE6FF16B5F
:1035F000A20EF06FF36BA30EF26FF56BF46FF76B27
:10360000A40EF66FF96BA50EF86FFB6BA60EFA6FA2
:10361000FD6BA70EFC6FFF6BFE6F0B01016BA80E1D
:10362000006F036BA90E026F056BAA0E046F076B88
:10363000066F096BAB0E086F0B6BAC0E0A6F0D6B50
:10364000AD0E0C6F0F6BAE0E0E6F116B106F136B18
:10365000AF0E126F156BB00E146F176BB10E166FA5
:10366000196B186F1B6BB20E1A6F1D6BB30E1C6FAC
:103670001F6BB40E1E6F216BB50E206F236B226F74
:10368000256BB60E246F276BB70E266F296BB80E0D
:10369000286F2B6B2A6F2D6BB90E2C6F2F6BBA0E08
:1036A0002E6F316BBB0E306F336B326F356BBC0ED0
:1036B000346F376BBD0E366F396BBE0E386F3B6B98
:1036C000BF0E3A6F3D6B3C6F3F6BC00E3E6F416B60
:1036D000C10E406F436BC20E426F456B446F476B28
:1036E000C30E466F496BC40E486F4B6BC50E4A6FD5
:1036F0004D6BC60E4C6F4F6B4E6F516BC70E506FBC
:10370000536BC80E526F556BC90E546F576B566F83
:10371000596BCA0E586F5B6BCB0E5A6F5D6BCC0E3C
:103720005C6F5F6B5E6F616BCD0E606F636BCE0E17
:10373000626F656BCF0E646F676BD00E666F696BDF
:10374000686F6B6BD10E6A6F6D6BD20E6C6F6F6BA7
:10375000D30E6E6F716B706F736BD40E726F756B6F
:10376000D50E746F776BD60E766F796BD70E786F38
:103770007B6B7A6F7D6BD80E7C6F7F6BD90E7E6F03
:10378000816BDA0E806F836B826F856BDB0E846FCB
:10379000876BDC0E866F896BDD0E886F8B6BDE0EA0
:1037A0008A6F8D6B8C6F8F6BDF0E8E6F916BE00E5F
:1037B000906F936BE10E926F956B946F976BE20E27
:1037C000966F996BE30E986F9B6BE40E9A6F9D6BEF
:1037D0009C6F9F6BE50E9E6FA16BE60EA06FA36BB7
:1037E000E70EA26FA56BE80EA46FA76BA66FA96B7F
:1037F000E90EA86FAB6BEA0EAA6FAD6BEB0EAC6F68
:10380000AF6BAE6FB16BEC0EB06FB36BED0EB26F12
:10381000B56BEE0EB46FB96B7E0EB86FBB6BBA6F43
:10382000BD6B7F0EBC6FBF6BBE6FC16B800EC06F78
:10383000C36BC26FC56B810EC46FC76BC66FC96B9C
:10384000820EC86FCB6BCA6FCD6B830ECC6FCF6B04
:10385000CE6FD16B840ED06FD36BD26FD56B850ECC
:10386000D46FD76BD66FD96B860ED86FDB6BDA6FE0
:10387000DD6B870EDC6FDF6BDE6FE16B880EE06F58
:10388000E36BE26FE56B890EE46FE76BE66FE96B64
:103890008A0EE86FEB6BEA6FED6B8B0EEC6FEF6BE4
:1038A000EE6FF16B8C0EF06FF36BF26FF56B8D0EAC
:1038B000F46FF76BF66FF96B8E0EF86FFB6BFA6FA8
:1038C000FD6B8F0EFC6FFF6BFE6F0C01016B900E9A
:1038D000006F036B026F056B910E046F076B066F31
:1038E000096B920E086F0B6B0A6F0D6B930E0C6FCA
:1038F0000F6B0E6F116B940E106F136B126F156BB5
:10390000950E146F176B166F196B960E186F1B6B55
:103910001A6F1D6B970E1C6F1F6B1E6F216B980E1D
:10392000206F236B226F256B990E246F276B266FF8
:10393000296B9A0E286F2B6B2A6F2D6B9B0E2C6FA9
:103940002F6B2E6F316B9C0E306F336B326F356B7C
:103950009D0E346F376B366F396B9E0E386F3B6B35
:103960003A6F3D6B9F0E3C6F3F6B3E6F416BA00EFD
:10397000406F436B426F456BA10E446F476B466FC0
:10398000496BA20E486F4B6B4A6F4D6BA30E4C6F89
:103990004F6B4E6F516BA40E506F536B526F556B44
:1039A000A50E546F576B566F596BA60E586F5B6B15
:1039B0005A6F5D6BA70E5C6F5F6B5E6F616BA80EDD
:1039C000606F636B626F656BA90E646F676B666F88
:1039D000696BAA0E686F6B6B6A6F6D6BAB0E6C6F69
:1039E0006F6B6E6F716BAC0E706F736B726F756B0C
:1039F000AD0E746F776B766F796BAE0E786F7B6BF5
:103A00007A6F7D6BAF0E7C6F7F6B7E6F816BB00EBC
:103A1000806F836B826F856BB10E846F876B866F4F
:103A2000896BB20E886F8B6B8A6F8D6BB30E8C6F48
:103A30008F6B8E6F916BB40E906F936B926F956BD3
:103A4000B50E946F976B966F996BB60E986F9B6BD4
:103A50009A6F9D6BB70E9C6F9F6B9E6FA16BB80E9C
:103A6000A06FA36BA26FA56BB90EA46FA76BA66F17
:103A7000A96BBA0EA86FAB6BAA6FAD6BBB0EAC6F28
:103A8000AF6BAE6FB16BBC0EB06FB36BB26FB56B9B
:103A9000BD0EB46FB96B6A0EB86FBB6BBA6FBD6BFE
:103AA0006B0EBC6FBF6BBE6FC16B6C0EC06FC36B18
:103AB0006D0EC26FC56BC46FC76B6E0EC66FC96BE0
:103AC000C86FCB6B6F0ECA6FCD6BCC6FCF6B700EA8
:103AD000CE6FD16BD06FD36B710ED26FD56BD46FAD
:103AE000D76B720ED66FD96B730ED86FDB6BDA6F34
:103AF000DD6B740EDC6FDF6BDE6FE16B750EE06FFC
:103B0000E36BE26FE56B760EE46FE76BE66FE96BF4
:103B1000770EE86FEB6BEA6FED6B780EEC6FEF6B87
:103B2000EE6FF16B790EF06FF36B7A0EF26FF56B4F
:103B3000F46FF76B7B0EF66FF96BF86FFB6B7C0E17
:103B4000FA6FFD6BFC6FFF6B7D0EFE6F0D01016B5D
:103B5000006F036B7E0E026F056B046F076B7F0EA9
:103B6000066F096B800E086F0B6B0A6F0D6B810E71
:103B70000C6F0F6B0E6F116B820E106F136B126F49
:103B8000156B830E146F176B166F196B840E186FFD
:103B90001B6B1A6F1D6B850E1C6F1F6B1E6F216BCD
:103BA000860E206F236B870E226F256B246F276B89
:103BB000880E266F296B286F2B6B890E2A6F2D6B51
:103BC0002C6F2F6B8A0E2E6F316B306F336B8B0E19
:103BD000326F356B346F376B8C0E366F396B8D0EE1
:103BE000386F3B6B3A6F3D6B8E0E3C6F3F6B3E6F99
:103BF000416B8F0E406F436B426F456B900E446F6D
:103C0000476B466F496B910E486F4B6B4A6F4D6B1C
:103C1000920E4C6F4F6B4E6F516B930E506F536BF8
:103C2000940E526F556B546F576B950E566F596BC0
:103C3000586F5B6B960E5A6F5D6B5C6F5F6B970E88
:103C40005E6F616B606F636B980E626F656B646F24
:103C5000676B990E666F696B9A0E686F6B6B6A6F14
:103C60006D6B9B0E6C6F6F6B6E6F716B9C0E706FDC
:103C7000736B726F756B9D0E746F776B766F796B6C
:103C80009E0E786F7B6B7A6F7D6B9F0E7C6F7F6B68
:103C90007E6F816BA00E806F836BA10E826F856B30
:103CA000846F876BA20E866F896B886F8B6BA30EF8
:103CB0008A6F8D6B8C6F8F6BA40E8E6F916B906F74
:103CC000936BA50E926F956B946F976BA60E966F84
:103CD000996BA70E986F9B6B9A6F9D6BA80E9C6F4C
:103CE0009F6B9E6FA16BA90EA06FA36BA26FA56BBC
:103CF000AA0EA46FA76BA66FA96BAB0EA86FAB6BD8
:103D0000AA6FAD6BAC0EAC6FAF6BAE6FB16BAD0E9F
:103D1000B06FB36BAE0EB26FB56BB46F0001120033
:023D2000FFD7CB
:020000040030CA
:0300010006170ED1
:020005008580F4
:060008000FC00FE00F40E5
:00000001FF
